:1000000012C03BC02BC02AC029C028C027C026C0B0
:1000100025C024C023C022C021C020C01FC01EC0D4
:100020001DC01CC01BC011241FBECFE5D4E0DEBF25
:10003000CDBF10E0A0E6B0E0E6EDF9E102C005902A
:100040000D92AA37B107D9F721E0AAE7B0E001C0C5
:100050001D92AD3CB207E1F7D3DBBBCCD1CF909181
:10006000600020E830E002C0359527958A95E2F7D8
:10007000209529232093600008951F920F920FB6B8
:100080000F9211242F933F934F938F939F938091BF
:100090007E00882329F080917D008F5F80937D0012
:1000A00080917C008F5F80937C0080917C008F3FEB
:1000B000B1F48BB78F7B8BBFA89AE0C690917D007F
:1000C00092FD806C87FF15C0A89A382F330F88E007
:1000D00090E020E8999BC6C60AB606FE0CC08AB717
:1000E00080648ABF8091600090917E00992351F3D3
:1000F000E5CFA898EACF999BB5C60AB606FCEFCF24
:10010000999BB0C60AB606FCEACF999BABC60AB665
:1001100006FCE5CF999BA6C60AB606FCE0CF999BE4
:10012000A1C60AB606FCDBCF999B9CC60AB606FCA4
:10013000D6CF999B97C60AB606FCD1CF999B92C69B
:100140000AB606FCCCCF999B8DC60AB606FCC7CF73
:10015000999B88C60AB606FCC2CF999B83C60AB68D
:1001600006FCBDCF999B7EC60AB606FCB8CF999B0C
:1001700079C60AB606FCB3CF999B74C60AB606FCCC
:10018000AECF999B6FC60AB606FCA9CF999B6AC6EB
:100190000AB606FCA4CF999B65C60AB606FC9FCF9B
:1001A000999B60C60AB606FC9ACF999B5BC60AB6B5
:1001B00006FC95CF999B56C60AB606FC90CF999B34
:1001C00051C60AB606FC8BCF999B4CC60AB606FCF4
:1001D00086CF999B47C60AB606FC81CF999B42C63B
:1001E0000AB606FC7CCF999B3DC60AB606FC77CFC3
:1001F000999B38C60AB606FC72CF999B33C60AB6DD
:1002000006FC6DCF999B2EC60AB606FC68CF999B5B
:1002100029C60AB606FC63CF999B24C60AB606FC1B
:100220005ECF999B1FC60AB606FC59CF999B1AC68A
:100230000AB606FC54CF999B15C60AB606FC4FCFEA
:10024000999B10C60AB606FC4ACF999B0BC60AB604
:1002500006FC45CF999B06C60AB606FC40CF999B83
:1002600001C60AB606FC3BCF999BFCC50AB606FC44
:1002700036CF999BF7C50AB606FC31CF999BF2C5DC
:100280000AB606FC2CCF999BEDC50AB606FC27CF13
:10029000999BE8C50AB606FC22CF999BE3C50AB62E
:1002A00006FC1DCF999BDEC50AB606FC18CF999BAC
:1002B000D9C50AB606FC13CF999BD4C50AB606FC6D
:1002C0000ECF999BCFC50AB606FC09CF999BCAC52C
:1002D0000AB606FC04CF999BC5C50AB606FCFFCE3C
:1002E000999BC0C50AB606FCFACE999BBBC50AB657
:1002F00006FCF5CE999BB6C50AB606FCF0CE999BD6
:10030000B1C50AB606FCEBCE999BACC50AB606FC95
:10031000E6CE999BA7C50AB606FCE1CE999BA2C57D
:100320000AB606FCDCCE999B9DC50AB606FCD7CE64
:10033000999B98C50AB606FCD2CE999B93C50AB67E
:1003400006FCCDCE999B8EC50AB606FCC8CE999BFD
:1003500089C50AB606FCC3CE999B84C50AB606FCBD
:10036000BECE999B7FC50AB606FCB9CE999B7AC5CD
:100370000AB606FCB4CE999B75C50AB606FCAFCE8C
:10038000999B70C50AB606FCAACE999B6BC50AB6A6
:1003900006FCA5CE999B66C50AB606FCA0CE999B25
:1003A00061C50AB606FC9BCE999B5CC50AB606FCE5
:1003B00096CE999B57C50AB606FC91CE999B52C51D
:1003C0000AB606FC8CCE999B4DC50AB606FC87CEB4
:1003D000999B48C50AB606FC82CE999B43C50AB6CE
:1003E00006FC7DCE999B3EC50AB606FC78CE999B4D
:1003F00039C50AB606FC73CE999B34C50AB606FC0D
:100400006ECE999B2FC50AB606FC69CE999B2AC56C
:100410000AB606FC64CE999B25C50AB606FC5FCEDB
:10042000999B20C50AB606FC5ACE999B1BC50AB6F5
:1004300006FC55CE999B16C50AB606FC50CE999B74
:1004400011C50AB606FC4BCE999B0CC50AB606FC34
:1004500046CE999B07C50AB606FC41CE999B02C5BC
:100460000AB606FC3CCE999BFDC40AB606FC37CE04
:10047000999BF8C40AB606FC32CE999BF3C40AB61F
:1004800006FC2DCE999BEEC40AB606FC28CE999B9D
:10049000E9C40AB606FC23CE999BE4C40AB606FC5E
:1004A0001ECE999BDFC40AB606FC19CE999BDAC40E
:1004B0000AB606FC14CE999BD5C40AB606FC0FCE2C
:1004C000999BD0C40AB606FC0ACE999BCBC40AB647
:1004D00006FC05CE999BC6C40AB606FC00CE999BC5
:1004E000C1C40AB606FCFBCD999BBCC40AB606FC87
:1004F000F6CD999BB7C40AB606FCF1CD999BB2C460
:100500000AB606FCECCD999BADC40AB606FCE7CD55
:10051000999BA8C40AB606FCE2CD999BA3C40AB66F
:1005200006FCDDCD999B9EC40AB606FCD8CD999BEE
:1005300099C40AB606FCD3CD999B94C40AB606FCAE
:10054000CECD999B8FC40AB606FCC9CD999B8AC4AF
:100550000AB606FCC4CD999B85C40AB606FCBFCD7D
:10056000999B80C40AB606FCBACD999B7BC40AB697
:1005700006FCB5CD999B76C40AB606FCB0CD999B16
:1005800071C40AB606FCABCD999B6CC40AB606FCD6
:10059000A6CD999B67C40AB606FCA1CD999B62C4FF
:1005A0000AB606FC9CCD999B5DC40AB606FC97CDA5
:1005B000999B58C40AB606FC92CD999B53C40AB6BF
:1005C00006FC8DCD999B4EC40AB606FC88CD999B3E
:1005D00049C40AB606FC83CD999B44C40AB606FCFE
:1005E0007ECD999B3FC40AB606FC79CD999B3AC44F
:1005F0000AB606FC74CD999B35C40AB606FC6FCDCD
:10060000999B30C40AB606FC6ACD999B2BC40AB6E6
:1006100006FC65CD999B26C40AB606FC60CD999B65
:1006200021C40AB606FC5BCD999B1CC40AB606FC25
:1006300056CD999B17C40AB606FC51CD999B12C49E
:100640000AB606FC4CCD999B0DC40AB606FC47CDF4
:10065000999B08C40AB606FC42CD999B03C40AB60E
:1006600006FC3DCD999BFEC30AB606FC38CD999B8E
:10067000F9C30AB606FC33CD999BF4C30AB606FC4F
:100680002ECD999BEFC30AB606FC29CD999BEAC3F0
:100690000AB606FC24CD999BE5C30AB606FC1FCD1D
:1006A000999BE0C30AB606FC1ACD999BDBC30AB638
:1006B00006FC15CD999BD6C30AB606FC10CD999BB6
:1006C000D1C30AB606FC0BCD999BCCC30AB606FC77
:1006D00006CD999BC7C30AB606FC01CD999BC2C340
:1006E0000AB606FCFCCC999BBDC30AB606FCF7CC47
:1006F000999BB8C30AB606FCF2CC999BB3C30AB661
:1007000006FCEDCC999BAEC30AB606FCE8CC999BDF
:10071000A9C30AB606FCE3CC999BA4C30AB606FC9F
:10072000DECC999B9FC30AB606FCD9CC999B9AC391
:100730000AB606FCD4CC999B95C30AB606FCCFCC6E
:10074000999B90C30AB606FCCACC999B8BC30AB688
:1007500006FCC5CC999B86C30AB606FCC0CC999B07
:1007600081C30AB606FCBBCC999B7CC30AB606FCC7
:10077000B6CC999B77C30AB606FCB1CC999B72C3E1
:100780000AB606FCACCC999B6DC30AB606FCA7CC96
:10079000999B68C30AB606FCA2CC999B63C30AB6B0
:1007A00006FC9DCC999B5EC30AB606FC98CC999B2F
:1007B00059C30AB606FC93CC999B54C30AB606FCEF
:1007C0008ECC999B4FC30AB606FC89CC999B4AC331
:1007D0000AB606FC84CC999B45C30AB606FC7FCCBE
:1007E000999B40C30AB606FC7ACC999B3BC30AB6D8
:1007F00006FC75CC999B36C30AB606FC70CC999B57
:1008000031C30AB606FC6BCC999B2CC30AB606FC16
:1008100066CC999B27C30AB606FC61CC999B22C380
:100820000AB606FC5CCC999B1DC30AB606FC57CCE5
:10083000999B18C30AB606FC52CC999B13C30AB6FF
:1008400006FC4DCC999B0EC30AB606FC48CC999B7E
:1008500009C30AB606FC43CC999B04C30AB606FC3E
:100860003ECC999BFFC20AB606FC39CC999BFAC2D2
:100870000AB606FC34CC999BF5C20AB606FC2FCC0E
:10088000999BF0C20AB606FC2ACC999BEBC20AB629
:1008900006FC25CC999BE6C20AB606FC20CC999BA7
:1008A000E1C20AB606FC1BCC999BDCC20AB606FC68
:1008B00016CC999BD7C20AB606FC11CC999BD2C222
:1008C0000AB606FC0CCC999BCDC20AB606FC07CC36
:1008D000999BC8C20AB606FC02CC999BC3C20AB651
:1008E00006FCFDCB999BBEC20AB606FCF8CB999BD1
:1008F000B9C20AB606FCF3CB999BB4C20AB606FC91
:10090000EECB999BAFC20AB606FCE9CB999BAAC273
:100910000AB606FCE4CB999BA5C20AB606FCDFCB5F
:10092000999BA0C20AB606FCDACB999B9BC20AB679
:1009300006FCD5CB999B96C20AB606FCD0CB999BF8
:1009400091C20AB606FCCBCB999B8CC20AB606FCB8
:10095000C6CB999B87C20AB606FCC1CB999B82C2C3
:100960000AB606FCBCCB999B7DC20AB606FCB7CB87
:10097000999B78C20AB606FCB2CB999B73C20AB6A1
:1009800006FCADCB999B6EC20AB606FCA8CB999B20
:1009900069C20AB606FCA3CB999B64C20AB606FCE0
:1009A0009ECB999B5FC20AB606FC99CB999B5AC213
:1009B0000AB606FC94CB999B55C20AB606FC8FCBAF
:1009C000999B50C20AB606FC8ACB999B4BC20AB6C9
:1009D00006FC85CB999B46C20AB606FC80CB999B48
:1009E00041C20AB606FC7BCB999B3CC20AB606FC08
:1009F00076CB999B37C20AB606FC71CB999B32C263
:100A00000AB606FC6CCB999B2DC20AB606FC67CBD6
:100A1000999B28C20AB606FC62CB999B23C20AB6F0
:100A200006FC5DCB999B1EC20AB606FC58CB999B6F
:100A300019C20AB606FC53CB999B14C20AB606FC2F
:100A40004ECB999B0FC20AB606FC49CB999B0AC2B2
:100A50000AB606FC44CB999B05C20AB606FC3FCBFE
:100A6000999B00C20AB606FC3ACB999BFBC10AB619
:100A700006FC35CB999BF6C10AB606FC30CB999B98
:100A8000F1C10AB606FC2BCB999BECC10AB606FC59
:100A900026CB999BE7C10AB606FC21CB999BE2C104
:100AA0000AB606FC1CCB999BDDC10AB606FC17CB27
:100AB000999BD8C10AB606FC12CB999BD3C10AB642
:100AC00006FC0DCB999BCEC10AB606FC08CB999BC0
:100AD000C9C10AB606FC03CB999BC4C10AB606FC81
:100AE000FECA999BBFC10AB606FCF9CA999BBAC156
:100AF0000AB606FCF4CA999BB5C10AB606FCEFCA51
:100B0000999BB0C10AB606FCEACA999BABC10AB66A
:100B100006FCE5CA999BA6C10AB606FCE0CA999BE9
:100B2000A1C10AB606FCDBCA999B9CC10AB606FCA9
:100B3000D6CA999B97C10AB606FCD1CA999B92C1A5
:100B40000AB606FCCCCA999B8DC10AB606FCC7CA78
:100B5000999B88C10AB606FCC2CA999B83C10AB692
:100B600006FCBDCA999B7EC10AB606FCB8CA999B11
:100B700079C10AB606FCB3CA999B74C10AB606FCD1
:100B8000AECA999B6FC10AB606FCA9CA999B6AC1F5
:100B90000AB606FCA4CA999B65C10AB606FC9FCAA0
:100BA000999B60C10AB606FC9ACA999B5BC10AB6BA
:100BB00006FC95CA999B56C10AB606FC90CA999B39
:100BC00051C10AB606FC8BCA999B4CC10AB606FCF9
:100BD00086CA999B47C10AB606FC81CA999B42C145
:100BE0000AB606FC7CCA999B3DC10AB606FC77CAC8
:100BF000999B38C10AB606FC72CA999B33C10AB6E2
:100C000006FC6DCA999B2EC10AB606FC68CA999B60
:100C100029C10AB606FC63CA999B24C10AB606FC20
:100C20005ECA999B1FC10AB606FC59CA999B1AC194
:100C30000AB606FC54CA999B15C10AB606FC4FCAEF
:100C4000999B10C10AB606FC4ACA999B0BC10AB609
:100C500006FC45CA999B06C10AB606FC40CA999B88
:100C600001C10AB606FC3BCA999BFCC00AB606FC49
:100C700036CA999BF7C00AB606FC31CA999BF2C0E6
:100C80000AB606FC2CCA999BEDC00AB606FC27CA18
:100C9000999BE8C00AB606FC22CA999BE3C00AB633
:100CA00006FC1DCA999BDEC00AB606FC18CA999BB1
:100CB000D9C00AB606FC13CA999BD4C00AB606FC72
:100CC0000ECA999BCFC00AB606FC09CA999BCAC036
:100CD0000AB606FC04CA999BC5C00AB606FCFFC941
:100CE000999BC0C00AB606FCFAC9999BBBC00AB65C
:100CF00006FCF5C9999BB6C00AB606FCF0C9999BDB
:100D0000B1C00AB606FCEBC9999BACC00AB606FC9A
:100D1000E6C9999BA7C00AB606FCE1C9999BA2C087
:100D20000AB606FCDCC9999B9DC00AB606FCD7C969
:100D3000999B98C00AB606FCD2C9999B93C00AB683
:100D400006FCCDC9999B8EC00AB606FCC8C9999B02
:100D500089C00AB606FCC3C9999B84C00AB606FCC2
:100D6000BEC9999B7FC00AB606FCB9C9999B7AC0D7
:100D70000AB606FCB4C9999B75C00AB606FCAFC991
:100D8000999B70C00AB606FCAAC9999B6BC00AB6AB
:100D900006FCA5C9999B66C00AB606FCA0C9999B2A
:100DA00061C00AB606FC9BC9999B5CC00AB606FCEA
:100DB00096C9999B57C00AB606FC91C9999B52C027
:100DC0000AB606FC8CC9999B4DC00AB606FC87C9B9
:100DD000999B48C00AB606FC82C9999B43C00AB6D3
:100DE00006FC7DC9999B3EC00AB606FC78C9999B52
:100DF00039C00AB606FC73C9999B34C00AB606FC12
:100E00006EC9999B2FC00AB606FC69C9999B2AC076
:100E10000AB606FC64C9999B25C00AB606FC5FC9E0
:100E2000999B20C00AB606FC5AC9999B1BC00AB6FA
:100E300006FC55C9999B16C00AB606FC50C9999B79
:100E400011C00AB606FC4BC9999B0CC00AB606FC39
:100E500046C9999B07C00AB606FC41C981E0809348
:100E60007F000CC0422F432311F0A89A01C0A8981C
:100E700026950197009709F02DC9F0CF9F918F918A
:100E80004F913F912F910F900FBE0F901F9018958B
:100E90009B01285F3F4F90E8492F4823FB01419376
:100EA000BF019695E217F307B9F70895A82FBB275E
:100EB000A7FDB09520EC3DE54BD52FEF3FE740E097
:100EC00050E02AD5822F0895892B11F0CB01C7C895
:100ED0009091600020E830E002C0359527956A9532
:100EE000E2F7922B909360000895EF92FF920F9398
:100EF0001F93CF93DF937A01C82FD0E0022F10E029
:100F0000E0E8F0E0E01BF10BCE17DF0714F4CB01B3
:100F1000A6D800581F4F0C171D0744F4C701DF91D6
:100F2000CF911F910F91FF90EF9099C8DF91CF91D2
:100F30001F910F91FF90EF9008958F929F92AF9223
:100F4000BF92CF92DF92EF92FF920F931F93CF93B6
:100F5000DF934A016901C82FD0E010E080E8A82E95
:100F6000B12CC501801B910BC817D9074CF4CB01DC
:100F700076D8AE18B108CA15DB0514F4C6016FD8CF
:100F800000581F4F0C171D07BCF4C40168D8F12C82
:100F900080E8E80EF11CEC16FD0674F4C601DF9142
:100FA000CF911F910F91FF90EF90DF90CF90BF9066
:100FB000AF909F908F9053C8DF91CF911F910F9169
:100FC000FF90EF90DF90CF90BF90AF909F908F9069
:100FD0000895EF920F9320917A0030917B008091D9
:100FE000CB012130310509F447C02230310509F425
:100FF0008AC0232B09F0D2C0807160E070E090E0DD
:1010000063DF8091CB01887061E070E090E05CDF8D
:101010008091CB01807862E070E090E055DF8091B4
:10102000CB0163E070E0817090E04EDF8091CC01F5
:1010300064E070E0817090E047DF8091CC018270C5
:1010400065E070E090E040DF8091CC01887066E060
:1010500070E090E039DF8091CC01847067E070E04F
:1010600090E032DF28E347E050E066E070E08091F6
:10107000C5013BDF28E33FC0807160E070E090E095
:1010800023DF8091CB01887061E070E090E01CDF8D
:101090008091CB01807862E070E090E015DF809174
:1010A000CB0163E070E0817090E00EDF8091CC01B5
:1010B00064E070E0817090E007DF8091CC01827085
:1010C00065E070E090E000DF8091CC01887066E020
:1010D00070E090E0F9DE8091CC01847067E070E010
:1010E00090E0F2DE20E247E050E066E070E08091C0
:1010F000C501FBDE20E245E050E064E070E0809155
:10110000C601F3DE4BC0807160E070E090E0DCDE91
:101110008091CB01887061E070E090E0D5DE809135
:10112000CB01807862E070E090E0CEDE8091CB0170
:1011300063E070E0817090E0C7DE8091CC0164E0F4
:1011400070E0817090E0C0DE8091CC01827065E03B
:1011500070E090E0B9DE8091CC01887066E070E0CC
:1011600090E0B2DE8091CC01847067E070E090E0A6
:10117000ABDE90E4E92E00E221E030E047E050E011
:1011800066E070E08091C501D8DE21E030E045E006
:1011900050E064E070E08091C601CFDE8091CB0129
:1011A00085FF04C081E080937E0002C010927E0023
:1011B0000F91EF900895FC01E058FF4F9F01285FC9
:1011C0003F4F90E880E040814111892B3196969500
:1011D000E217F307C1F70895CF92DF92EF92FF92E3
:1011E0000F931F93CF93DF936B017A018C01EA0178
:1011F000CE018E199F098C159D0534F4C801DBDFE3
:101200008993085F1F4FF4CFDF91CF911F910F910A
:10121000FF90EF90DF90CF900895A598AD98BC9A7D
:10122000C49808950F931F93CF93DF93662309F417
:1012300061C077279B0143E0220F331F4A95E1F7F6
:101240002D32314004F5F0E0E0E040E050E02F2F97
:101250003E2F46175707D4F4D901189610E8FC0121
:10126000E40FF51F00810123E901C058DF4F088317
:101270002F5F3F4F16952A173B07A1F74F5F5F4F30
:10128000F22FE32FE4CF80E090E002C08F2F9E2F5B
:10129000009709F42FC0E0E8F0E0CF93DF93EF93DD
:1012A000FF930191002311F049F416C00000A59AA4
:1012B00019E00FD0A5980197A1F70EC0A59A11E0EB
:1012C00008D0A59815E005D000000000019749F767
:1012D00003C01A95F1F708950000FF91EF91DF9197
:1012E000CF91A59A11E0F5DFA5980FEF0A9511F0BF
:1012F0009D9BFCCFE0E8F0E0EF93FF9344270027AD
:101300000395A1F09D99FCCF08C004E6039572F007
:101310009D99FCCF439551F0019304E6039532F07B
:101320009D9BFCCF439511F00193EFCFFF91EF917F
:10133000842F90E00097C1F040FF16C0DF019D01AF
:101340007081618151E0761708F050E05D9332962C
:101350005A2F521B5417A0F32AE12A95F1F700C027
:1013600001979595879502C080E090E0DF91CF913D
:101370001F910F9108950F931F93CF93DF931F92A7
:10138000CDB7DEB7198261E070E0CE0101964ADF89
:10139000009751F1489759F580E090E00CDF082F55
:1013A00010E0102F002788E090E005DF9801282B3F
:1013B000C901292F33272F7033272830310571F0C9
:1013C00030F42530310599F481E090E015C02930E2
:1013D000310581F02B30310569F009C08032984029
:1013E00049F483E090E008C080E090E005C084E02C
:1013F00090E002C082E090E00F90DF91CF911F91CA
:101400000F910895009741F028E0E8EBF1E0DC014E
:1014100001900D922A95E1F788E0E8EBF1E0A0EB6E
:10142000B1E001900D928A95E1F788E090E008958F
:101430009093AF018093AE01089548E050E060EBD7
:1014400071E088EB91E0B8D20895BF92CF92DF921D
:10145000EF92FF920F931F93CF93DF93CDB7DEB739
:1014600029970FB6F894DEBF0FBECDBF198661E095
:1014700070E0CE010996D6DE883111F081E0A5C07A
:1014800080E4898383E08A8321E08091AE0190919A
:10149000AF01892B09F420E02B8363E070E0CE01DB
:1014A0000196C0DE803451F780E090E084DEB82EF3
:1014B00088E090E080DEC82E80E190E07CDED82ECF
:1014C00088E190E078DEE82E80E290E074DEF82E8D
:1014D00088E290E070DE082F80E390E06CDE182F49
:1014E00088E390E068DE20E030E090E060E170E0CA
:1014F000AB2DB0E0E1E0AB01022E02C0559547955F
:101500000A94E2F74A235B23452B39F04E2F022E33
:1015100001C0440F0A94EAF701C040E0942B2F5F0A
:101520003F4F2530310539F7C6FC02C030E001C01D
:1015300030E2932BC5FC02C030E001C030E4392B0F
:10154000C4FC02C020E001C020E8A32FA22B20E0B1
:1015500030E090E068E070E0EC2DF0E0B1E0AB014D
:10156000022E02C0559547950A94E2F74E235F2359
:10157000452B39F04B2F022E01C0440F0A94EAF795
:1015800001C040E0942B2F5F3F4F2430310539F7E5
:101590002091AC013091AD01232B11F01FE78FE7B3
:1015A000D092B801E094E092B901F092BA010095AE
:1015B0000093BB0110951093BC0180958093BD01F1
:1015C000A093BE019093BF0180E029960FB6F894D6
:1015D000DEBF0FBECDBFDF91CF911F910F91FF9066
:1015E000EF90DF90CF90BF9008952FDF91E08111B1
:1015F00090E0892F089529DF811111C088E090E0E3
:10160000DADD8670863039F481E090E09093AD01A8
:101610008093AC0108951092AD011092AC01089531
:1016200081E690E008950F931F93CF93DF93CDB79A
:10163000DEB7C254D1090FB6F894DEBF0FBECDBFDE
:10164000FE013196982FEF93FF9300E8192F102396
:10165000D1F0000068C0A59A000000000000000062
:10166000000000000000000000000000000000007A
:1016700000000000A5983CE03A95F1F7000000005A
:10168000069581F0E3CFA59A3FE03A95F1F7000087
:10169000A598000000000000000000000000069572
:1016A00009F0D4CFA5980000000000000000000061
:1016B000000000000000A59A0000000000000000EB
:1016C000000000000000000000000000000000001A
:1016D00000000000A59830E20FEF0A9511F113B356
:1016E0001072D9F7000000000000000000000000A8
:1016F00000000000000000000000000000000000EA
:10170000000023B3207221933A9539F00FEF0A9528
:1017100041F023B3207201F7FACF882704C0832F4A
:1017200002C088278095FF91EF9123968FAF239772
:1017300023962FAD239781E090E02F3F11F080E0BA
:1017400090E0919581959109CE5BDF4F0FB6F894AB
:10175000DEBF0FBECDBFDF91CF911F910F910895D6
:101760001FBC83E08EBD1DBC1CBC1092C0018DE16E
:1017700099E09093C2018093C101089508B602FEDA
:1017800004C088B7846088BF17C08CB59DB5853A02
:1017900026E09207B8F08C382AE09207D8F0875EEE
:1017A00093409093C2018093C1018091C1019091B7
:1017B000C201843A964030F48DE199E09093C201E1
:1017C0008093C1011DBC1CBC88B7846088BF109287
:1017D000C00108958DE199E0E4CF8091C0018111AD
:1017E0000DC02CB53DB58091C1019091C201281763
:1017F000390720F081E08093C001089580E00895CA
:101800000FDF9093C4018093C30111BA8FEF82BBA5
:1018100017BA88BB90E297BBC59891E094BB85BB93
:1018200085B7836085BF8BB780648BBF8BB78F779D
:101830008BBFF3DCE091C301F091C4010484F58512
:10184000E02D09952FEF89E698E1215080409040E6
:10185000E1F700C00000E091C301F091C4010684EB
:10186000F785E02D0995E091C301F091C40102884C
:10187000F389E02D60E070E085EC91E0099520911E
:10188000CB0124FF06C082E090E090937B00809320
:101890007A0023FF06C081E090E090937B00809364
:1018A0007A005EDF789480917F00882319F010928F
:1018B0007F0064DF92DF811104C080917C008F3F44
:1018C00091F7E091C301F091C4010684F785E02D02
:1018D0000995E091C301F091C4010088F189E02DE0
:1018E00080E090E00995882369F0E091C301F091D0
:1018F000C4010288F389E02D60E070E085EC91E09E
:10190000099567DB80917C008F3F19F48BB7806469
:101910008BBF10927C00C7CF052E97FB16F4009466
:101920000FD057FD05D01AD007FC02D046F408C0EE
:1019300050954095309521953F4F4F4F5F4F0895FB
:1019400090958095709561957F4F8F4F9F4F08952B
:1019500027D0B7FF0895821B930B0895A1E21A2E9A
:10196000AA1BBB1BFD010DC0AA1FBB1FEE1FFF1F43
:10197000A217B307E407F50720F0A21BB30BE40B93
:10198000F50B661F771F881F991F1A9469F76095DA
:101990007095809590959B01AC01BD01CF01089594
:1019A000A29FB001B39FC001A39F01D0B29F700D51
:1019B000811D1124911D0895FB01DC0104C08D914E
:1019C0000190801921F441505040C8F7881B990BB1
:0619D0000895F894FFCF1A
:1019D600FF010000000000000000000000FB0A25D7
:0A19E6000A1D0A020A180AF50A0099
:00000001FF
